:100000002BC038C037C036C035C034C033C032C052
:100010004DC030C04E4C4954452062792044724A4C
:100020006F6E65732040204275646765744C696724
:100030006874466F72756D2E636F6D202832303193
:1000400033290003145CFF0803FF5214080408144A
:100050005CFF04FF5214080011241FBECFE9CDBF7E
:1000600010E0A0E6B0E001C01D92A536B107E1F7AF
:1000700066D0CAC0C5CF282F90916100892F8F5FAD
:1000800080936100803210F01092610080916100D5
:100090008EBB2DBB84E08CBBE19AE199FECF9EBB69
:1000A00084E18CBBE19AE199FECF08951F920F92F3
:1000B0000FB60F9211242F933F934F935F936F933B
:1000C0007F938F939F93AF93BF93EF93FF93809111
:1000D00063008F3F19F08F5F80936300809163000E
:1000E000873039F4B39902C081E002C08091640086
:1000F000C2DF369A3699FECF85B18D3768F480918C
:1001000062008F5F80936200893040F080916000D0
:1001100086958C5F8093600010926200FF91EF9152
:10012000BF91AF919F918F917F916F915F914F910F
:100130003F912F910F900FBE0F901F9018951F9316
:10014000CF93DF9382E087BB89EF88BB83E481BDD7
:10015000789485B7877C806285BF83E28FBD81E01C
:1001600083BF479A81E687B984EC86B9B09902C00B
:1001700082E001C080E0B49B8F5F90E065E070E0BA
:1001800031D0EC01FC01ED5BFF4F949110926100C6
:1001900080E08EBBE09A1DB31F3F19F48F5F803261
:1001A000C0F38093610080916100803219F4109255
:1001B000610011E0911708F411E010936400812FA1
:1001C0008F5F981708F481E056DFC10FD11DCD5B1A
:1001D000DF4FFE018491809360008091600089BDB3
:1001E0008895FBCF5527002480FF02C0060E571FBD
:1001F000660F771F6115710521F096958795009719
:0C02000099F7952F802D0895F894FFCFFA
:00000001FF
